:020000040000FA
:020000000428D2
:08000800FF30A200FF30A3004D
:10001000FF30A400FF30A5000F30A600A901AA01FF
:1000200024138A150A123822A4178A150A123522B7
:100030008A150A126622203098000D3099008A1520
:100040000A126922903098001A081A081A0800301B
:100050009900F801FE01FC01FA01F701FD01FB0125
:10006000F901FF308A150A1251228A150A12D72087
:1000700023108A150A124722A3108A150A12442255
:1000800023118A150A124122A3118A150A123E224F
:1000900023128A150A123B22A2148A150A124A2236
:1000A00027128A150A121C2227148A150A122822DE
:1000B000A7108A150A12252227118A150A12222250
:1000C000A7118A150A121F2201308A150A12A621C9
:1000D00027108A150A122822A7148A150A12252227
:1000E00027118A150A122222A7118A150A121F2225
:1000F00001308A150A12A62127108A150A12282211
:10010000A7108A150A12252227158A150A122222FB
:10011000A7118A150A121F2201308A150A12A62178
:1001200027108A150A122822A7108A150A122522DA
:1001300027118A150A122222A7158A150A121F22D0
:1001400001308A150A12A621A7118A150A121F2248
:100150008A150A1205218A150A12E52002308A152D
:100160000A12DF204F308A150A1230214E308A15CC
:100170000A12302134308A150A12302149308A158A
:100180000A12302159308A150A12302120308A157E
:100190000A12302132308A150A12302130308A1585
:1001A0000A12302130308A150A12302135308A1572
:1001B0000A12302140308A150A12DF2052308A1587
:1001C0000A1230214F308A150A12302156308A1512
:1001D0000A12302145308A150A12302152308A1510
:1001E0000A12302142308A150A1230214F308A1506
:1001F0000A12302158308A150A12302120308A150F
:100200000A12302176308A150A12302132308A15CE
:100210000A12302134308A150A12302120308A1512
:100220000A12302120308A150A12302144308A15F2
:100230000A12302157308A150A12302101308A15EE
:100240000A129D2101308A150A129D2120118A115E
:100250000A12851C2C2920158A110A12201D7B29BF
:100260008A150A12E52040308A150A12DF20203054
:100270008A150A12302120308A150A1230214530A1
:100280008A150A12302158308A150A12302150304E
:100290008A150A12302145308A150A12302152304F
:1002A0008A150A12302149308A150A1230214D3040
:1002B0008A150A12302145308A150A1230214E3033
:1002C0008A150A12302154308A150A123021413021
:1002D0008A150A1230214C308A150A12302120303A
:1002E0008A150A12302120308A150A123021013075
:1002F0008A150A129D2127148A150A1228228A15A6
:100300000A12E520B601D001A011A01400308A1510
:100310000A12DF208A110A12A01992298A110A12E0
:10032000A01895298A110A12D6298A150A122620A0
:100330005A08AB002B08243C8A110A120319A4297D
:100340008A110A12A018A7298A110A12AF298A1540
:100350000A128C205A08AB008A110A129A298A11B3
:100360000A12A01CD3298A150A128C205A08AB0045
:100370008A150A128C205A08AC008A150A128C20A1
:100380005A08AD008A150A128C205A08AE008A1548
:100390000A128C205A08AF002F08433C8A110A1217
:1003A000031DD329A0158A110A128A298A110A125B
:1003B000A01CF6298A110A12A01DF6298A150A1214
:1003C0008C205A08AB0040307D028A110A12031CAF
:1003D000EC298A110A12F6298A150A128C205A0869
:1003E0008A150A127C208A110A12E3298A110A123C
:1003F000A01C6C2E8A110A12A01D6C2E8A150A12DE
:100400006D205E08B9008A150A126D205E08BA00D8
:100410008A150A126D205E08BB008A150A126D202B
:100420005E08BC008A150A126D205E08BD008A15A0
:100430000A126D205E08BE000230BE0730303E0258
:10044000093C8A110A120318292A0A303E02BE000A
:10045000BD0A30303D02053C8A110A120318332AC6
:100460003030BD00BC0A30303C02093C8A110A120F
:1004700003183E2A0A303C02BC00BB0A30303B0263
:10048000053C8A110A120318482A3030BB00BA0A08
:100490008A150A126D205E082C3C8A110A12031973
:1004A000542A8A110A12482A8A150A126D205E08F7
:1004B000413C8A110A12031D612A20168A110A1270
:1004C000622A20128A150A126D205E082C3C8A11BD
:1004D0000A1203196E2A8A110A12622A8A150A124E
:1004E0006D205E08C5008A150A126D205E08C600E0
:1004F0008A150A126D205E08C7008A150A126D203F
:100500005E08C8008A150A126D205E08C9008A15A7
:100510000A126D205E08C9008A150A126D205E0855
:100520002C3C8A110A120319982A8A110A128C2A61
:100530008A150A126D205E082C3C8A110A120319D2
:10054000A42A8A110A12982A8A150A126D205E08B6
:10055000CA008A150A126D205E08CB008A150A129D
:100560006D205E08CC008A150A126D205E08CD0051
:100570008A150A126D205E08CE008A150A126D20B7
:100580005E082C3C8A110A120319C92A8A110A1220
:10059000BD2A8A150A126D205E08CF008A150A123C
:1005A0006D205E082C3C8A110A120319DA2A8A117E
:1005B0000A12CE2A8A150A126D205E082C3C8A1176
:1005C0000A120319E62A8A110A12DA2A8A150A126D
:1005D0006D205E082C3C8A110A120319F22A8A1136
:1005E0000A12E62A8A150A126D205E08BF008A15D3
:1005F0000A126D205E08C0008A150A126D205E087E
:10060000C1008A150A126D205E08C2008A150A12FE
:100610006D205E08C3008A150A126D205E08C400B2
:100620004F08453C8A110A12031D3E2B30304A0206
:10063000F3006430F4008A150A12B022DC005C0872
:10064000DB0030304C02DD0030304B02F3000A306A
:10065000F4008A150A12B022DE005E085D075B070F
:10066000F1001430F2008A150A129722DA005A08B3
:10067000093E413EB0008A110A12632B30304A0213
:10068000F3006430F4008A150A12B022E100610818
:10069000E00030304C02E20030304B02F3000A3010
:1006A000F4008A150A12B022E300630862076007AB
:1006B000F1001430F2008A150A129722DF005F0859
:1006C000083C413EB00030304602E0003030450288
:1006D000F3000A30F4008A150A12B022E100610822
:1006E0006007F1000A30F2008A150A129722DF0033
:1006F0005F08093E413EB1004F08453C8A110A128D
:10070000031DB12B30304A02F3006430F4008A1527
:100710000A12B022E5006508E40030304C02E60021
:1007200030304B02F3000A30F4008A150A12B0226E
:10073000E700670866076407F1001430F2008A15C5
:100740000A128022E3006308EE000130EF008A15F0
:100750000A126C22E2006208303EB2008A110A12CC
:10076000DE2B30304A02F3006430F4008A150A129E
:10077000B022EB006B08EA0030304C02EC00303065
:100780004B02F3000A30F4008A150A12B022ED0081
:100790006D086C076A07F1001430F2008A150A121E
:1007A0008022E9006908EE000130EF008A150A1284
:1007B0006C22E8006808093C303EB2004608B300ED
:1007C0004F08453C8A110A12031D232C30304C027D
:1007D0000139003C8A110A12031D082C30304E02E8
:1007E000E90030304D02F3000A30F4008A150A1295
:1007F000B022EA006A086907F1000530F2008A15A4
:100800000A129722E8006808B8008A110A12202C00
:1008100030304E02EC0030304D02F3000A30F4006C
:100820008A150A12B022ED006D086C073C3EF100FB
:100830000530F2008A150A129722EB006B08B80007
:100840008A110A125E2C30304C020139013C8A11A7
:100850000A12031D462C30304E02EC0030304D029F
:10086000F3000A30F4008A150A12B022ED006D0878
:100870006C07F1000530F2008A150A129722EB008E
:100880006B080B3CB8008A110A125E2C30304E0205
:10089000EF0030304D02F3000A30F4008A150A12DE
:1008A000B022F00070086F07F1000530F2008A15E1
:1008B0000A129722EE006E08173CB8003808203E56
:1008C000413EB40030304802EC0030304702F300C3
:1008D0000A30F4008A150A12B022ED006D086C0788
:1008E000F1000530F2008A150A129722EB006B081E
:1008F000B5000310350D413EB50030304802EF0021
:1009000030304702F3000A30F4008A150A12B02290
:10091000F00070086F07F1000530F2008A150A1226
:100920008022EE006E08B8003808023C8A110A12D4
:1009300003189B2CB50A3808023C8A110A12031DC1
:10094000A82C4908053C8A110A120318A82CB50ADC
:100950002030B50740308A150A12DF2039088A1581
:100960000A1230213A088A150A1230213A308A15C3
:100970000A1230213B088A150A1230213C088A15D8
:100980000A12302120308A150A12302120308A15AF
:100990000A12302120308A150A12302120308A159F
:1009A0000A1230218A110A122019F52C20308A15DA
:1009B0000A12302130088A150A12302131088A15AE
:1009C0000A12302132088A150A12302133088A159A
:1009D0000A12302134088A150A12302135088A1586
:1009E0000A1230218A110A12D72DD0088A110A1250
:1009F000031D192D3F308A150A12302130088A153F
:100A00000A12302131088A150A12302132088A155B
:100A10000A12302133088A150A12302134088A1547
:100A20000A12302135088A150A1230218A110A1259
:100A3000D72DB6088A110A12031D472D033059021B
:100A40008A110A1203182B2D20308A150A12302120
:100A50008A110A122F2D3F308A150A1230213008D0
:100A60008A150A12302131088A150A1230213208FB
:100A70008A150A12302133088A150A1230213408E7
:100A80008A150A12302135088A150A1230213608D3
:100A9000053C8A110A12031D762D033059028A1172
:100AA0000A1203185A2D20308A150A1230218A1191
:100AB0000A125E2D3F308A150A12302151088A151C
:100AC0000A12302152088A150A12302120308A1564
:100AD0000A12302153308A150A12302141308A150A
:100AE0000A12302154308A150A1230213608083C87
:100AF0008A110A12031DA52D033059028A110A1208
:100B00000318892D20308A150A1230218A110A1201
:100B10008D2D3F308A150A12302141308A150A1274
:100B2000302153088A150A12302154088A150A12F6
:100B3000302155088A150A12302156088A150A12E2
:100B400030216D308A150A12302136080B3C8A118B
:100B50000A12031DD62D033059028A110A120318F6
:100B6000B82D20308A150A1230218A110A12BC2DA4
:100B70003F308A150A12302148308A150A12302176
:100B800044308A150A1230214F308A150A1230215A
:100B900050308A150A12302157088A150A1230215E
:100BA00058088A150A123021FF30B600B60A003004
:100BB0008A150A12DF203F088A150A1230214008E0
:100BC0008A150A1230212F308A150A123021410865
:100BD0008A150A12302142088A150A123021303053
:100BE0003C020139013C8A110A12031D0E2E2030ED
:100BF0008A150A1230214F308A150A1230214430EA
:100C00008A150A12302144308A150A123021203008
:100C10008A150A1230218A110A12222E20308A15D2
:100C20000A12302145308A150A12302156308A15B1
:100C30000A12302145308A150A1230214E308A15A9
:100C40000A1230218A110A12201E492E27158A15F0
:100C50000A122222A7118A150A121F220B308A15A6
:100C60000A12DF203B088A150A1230213C088A1537
:100C70000A1230213A308A150A1230213D088A15AD
:100C80000A1230213E088A150A1230218A110A12EE
:100C9000692E27118A150A122222A7158A150A120F
:100CA0001F220B308A150A12DF2049308A150A12DA
:100CB00030214E308A150A12302156308A150A1218
:100CC000302141308A150A1230214C308A150A121F
:100CD00030218A110A12942E8A110A12A018942E19
:100CE00048308A150A12DF204E308A150A12302148
:100CF0004F308A150A12302120308A150A1230210D
:100D000047308A150A12302150308A150A123021D4
:100D100053308A150A12302120308A150A123021E8
:100D200020308A150A123021FD01FE01A7148A1510
:100D30000A12252201308A150A12AF21A7108A153E
:100D40000A122522B6088A150A12031D20288A15C0
:100D50000A12201D2028A011A0148A110A12A0191D
:100D6000B52E8A110A12A018B82E8A110A12F92E6D
:100D70008A150A1226205A08AB002B08243C8A1137
:100D80000A120319C72E8A110A12A018CA2E8A1134
:100D90000A12D22E8A150A128C205A08AB008A1128
:100DA0000A12BD2E8A110A12A01CF62E8A150A12EA
:100DB0008C205A08AB008A150A128C205A08AC0005
:100DC0008A150A128C205A08AD008A150A128C2046
:100DD0005A08AE008A150A128C205A08AF002E0855
:100DE000473C8A110A12031DF62EA0158A110A1219
:100DF000AD2E8A110A12A01C192F8A110A12A01DE9
:100E0000192F8A150A128C205A08AB0040307D0237
:100E10008A110A12031C0F2F8A110A12192F8A1520
:100E20000A128C205A088A150A127C208A110A128A
:100E3000062F8A110A12A01CEE2F8A110A12A01D79
:100E4000EE2FB701053037028A110A12031C2B2F2F
:100E50008A110A123B2F8A150A126D205E082C3C5B
:100E60008A110A120319372F8A110A122B2FB70A77
:100E70008A110A12222F8A150A126D205E08DA00E2
:100E800030305A02D0008A150A126D205E08D10057
:100E90008A150A126D205E08D1008A150A126D208B
:100EA0005E08D200D0088A110A120319EB2F8A15A6
:100EB0000A126D205E08D3008A150A126D205E08A2
:100EC000D7008A150A126D205E08D80058082E3CFB
:100ED0008A110A12031D702F5708D8003030D7002E
:100EE0005708303C8A110A12031D842F5808393CD8
:100EF0008A110A12031D832F3030D8003130D700F9
:100F00008A110A12842FD80A30305802DB003030A0
:100F10005702F3000A30F4008A150A12B022DC00EE
:100F20005C085B07D9008A150A126D205E082C3C0C
:100F30008A110A1203199F2F8A110A12932F8A15F8
:100F40000A126D205E08D3008A150A126D205E0811
:100F5000D4008A150A126D205E08D5008A150A127F
:100F60006D205E08D60053082E3C8A110A12031D1C
:100F7000C12F2030D6002030D5002030D4002030C2
:100F8000D30054082E3C8A110A12031DCF2F530898
:100F9000D6002030D5002030D4002030D3005508B2
:100FA0002E3C8A110A12031DDD2F5408D600530867
:100FB000D5002030D4002030D30056082E3C8A11B2
:100FC0000A12031DEB2F5508D6005408D50053080C
:100FD000D4002030D3008A150A1212288A150A126A
:100FE000A018122848308A150A12DF204E308A15C0
:100FF0000A1230214F308A150A12302147308A15E3
:101000000A12302150308A150A12302153308A15C5
:101010000A12302120308A150A12302120308A1518
:101020000A123021FD01FE0127168A150A121C2220
:1010300001308A150A12AF2127128A150A121C22C2
:101040008A110A1284298A150A122328DA00FF302D
:10105000DB00FF30DC00A0108A150A12AB205D080F
:10106000DA008A150A12201F3928A0148A150A12DC
:101070006C28DB088A150A12031942288A150A12FD
:10108000A01C45288A150A126C28DC088A150A1249
:1010900003194E288A150A12A01C51288A150A1213
:1010A000642801305C02DC008A150A12AB205D085E
:1010B000DA008A150A12201F6128A0148A150A1264
:1010C0006C288A150A12452801305B02DB00FF30CC
:1010D000DC008A150A12392808004F307E028A1572
:1010E0000A12031C7428FE017E08A03E84008313AC
:1010F000FE0A0008DE000800DB004F307D028A1582
:101100000A12031C8428FD017D08A03E840083137D
:101110005B088000FD0A0800DA0098189A28181960
:10112000A4288C1E8D288B138B1B93281A088B17D1
:10113000DA00AA288B138B1B9A2818121A081A088F
:101140001A0818168B178D288B138B1BA4281A08C6
:101150008B178D280800DD008A150A128C1EB42812
:10116000A0178A150A12B528A0139818C0281819B4
:10117000CA288B138B1BB9281A088B17DD00D028BF
:101180008B138B1BC02818121A081A081A08181675
:101190008B17B5288B138B1BCA281A088B17B528F9
:1011A00020138A150A12A01FD628201708008A15B6
:1011B0000A12662287309F008A150A12692AF100F6
:1011C0007108803E8A150A123E2908308A150A12D3
:1011D0003E2101308A150A123E21C8308A150A12B2
:1011E000E42102308A150A123E21C8308A150A12FB
:1011F000E42106308A150A123E210C308A150A12A3
:101200003E21C8308A150A12E4298A150A1295214E
:1012100064308A150A12B821A8108A150A121922F8
:1012200003308A150A12542132308A150A12F82125
:1012300003308A150A12542132308A150A12F82115
:1012400003308A150A12542132308A150A12F82105
:1012500032308A150A123E2128308A150A123E2998
:10126000F100A8148A150A121922710E0F398A1575
:101270000A12542171088A150A125429F200A81082
:101280008A150A121922720E0F398A150A12542170
:101290000D308A150A12C12172088A150A125421CA
:1012A0000D308A150A12C129F30028118A150A1275
:1012B0001622A8158A150A1213222812730801395A
:1012C000003C8A150A120318662928168A150A1284
:1012D0001022A81273080239003C8A150A1203185A
:1012E0007229A8168A150A120D22281373080439C8
:1012F000003C8A150A1203187E2928178A150A123B
:101300000A22A81373080839003C8A150A12031828
:101310008A29A8178A150A120722A8118A150A1203
:10132000132219308A150A12E42900308A150A128C
:101330004D2200308A150A122B2AAB002B08F4002C
:101340006430F50064308A150A12CA29AB002B08F4
:10135000F4006430F50014308A150A12CA29DA0044
:101360005A08F4006430F5000A308A150A12CA29B6
:10137000AB002B08F4000A30F50001308A150A1280
:10138000CA29F3007308F4000130F50001308A1512
:101390000A12CA29F600FF30F7007508F900740830
:1013A000F80017308A150A1277070318D4298A150E
:1013B0000A12F80BD1298A150A12F90BCF298A15BE
:1013C0000A12F60BCD290800F4007408F500F508A0
:1013D0008A150A12031DEF298A150A12F7290A3005
:1013E0008A150A12F821F5038A150A12E72908005E
:1013F000F600F430F700FC30F8008A150A1276087F
:101400007707031C003478070318032A08008A159D
:101410000A122F2A8A150A122F2A8A150A122F2A2F
:101420008A150A122F2A8A150A122F2A8A150A12D9
:101430002F2A8A150A122F2A8A150A12322A8A1589
:101440000A12322A8A150A12322A8A150A12322AF6
:101450008A150A12322AA8008A150A122F2A280889
:10146000880008002708860008008A150A125D2AED
:101470008A150A125D2A8A150A12602A8A150A122A
:10148000602A8A150A12602A8A150A12602A8A15A9
:101490000A12602A8A150A12632AA5008A150A12FE
:1014A000552AA2008A150A12632A25088A150A12EB
:1014B000662288008A150A12692A24086700080033
:1014C000230866000800220865000800831603133D
:1014D0000800831203130800EF006F08003C8A1510
:1014E0000A12031C762A8A150A127E2A0310EE0CB1
:1014F00001306F02EF008A150A126D2A6E0808008B
:10150000F200F2088A150A120319952A720871026C
:101510008A150A1203188F2A8A150A12952A720848
:101520007102F1008A150A12862A71080800F20079
:10153000F301F2088A150A120319AE2A7208710221
:101540008A150A120318A72A8A150A12AE2A7208E7
:101550007102F100F30A8A150A129E2A7308080024
:10156000F400F5017408003C8A150A12031CBB2A1A
:101570008A150A12C32A7308F50701307402F400B1
:0A1580008A150A12B22A7508080045
:02400E00723FFF
:00000001FF
